:200000000C946E010C9496010C9496010C9496010C9496010C9496010C9496010C94960150
:200020000C9496010C9496010C941B050C94A6050C9496010C9496010C9496010C9496016B
:200040000C9496010C9496010C9496010C9496010C9496010C9496010C9496010C94B201CC
:200060000C9496010C9496010C9496010C9496010C9496010C9496010C9496010C949601C8
:200080000C9496010C9496010C9496010C9496010C9496010C9496010C9496010C949601A8
:2000A0000C9496010C9496010C94960100000000240027002A002D003000000000002500A4
:2000C00028002B002E003100000000002300260029002C002F00040404040403040502027D
:2000E0000202040302020202060606060606040402020204040802011040804010204080A8
:200100004080080204018040201002011080102040400000000200080E0000030401000BB2
:200120000000070605040100080A0B0C0D09040309042203410072006400750069006E00CD
:200140006F0020004D006900630072006F00200020002000180341007200640075006900A6
:200160006E006F0020004C004C004300120100020000004041233580000101020001120121
:200180000002020000404123358000010102000100C18081C1080B00020202010009040053
:2001A000000102020000052400100105240101010424020605240600010705810310004094
:2001C00009040100020A000000070502024000000705830240000005010902A1010901A186
:2001E000008501050919012903150025019503750181029501750581030501093009310943
:20020000381581257F750895038106C0C005010906A1018502050719E029E715002501754D
:20022000019508810295017508810395067508150025650507190029658100C0090402004C
:2002400001030000000921010100012265000705840340000100000000000000002A2B2895
:200260000000000000000000000000000000000000000000002C9EB4A0A1A2A434A6A7A553
:20028000AE362D3738271E1F20212223242526B333B62EB7B89F8485868788898A8B8C8D58
:2002A0008E8F909192939495969798999A9B9C9D2F3130A3AD350405060708090A0B0C0D7C
:2002C0000E0F101112131415161718191A1B1C1DAFB1B0B5000057043907370811241FBE15
:2002E000CFEFDAE0DEBFCDBF11E0A0E0B1E0E4EEF2E102C005900D92AA32B107D9F711E06B
:20030000AAE2B1E001C01D92AB39B107E1F712E0CCEDD2E004C02297FE010E946C09C63DE9
:20032000D107C9F70E9491030C9470090C9400008DE061E00E945E0368EE73E080E090E00C
:200340000E94FA018DE060E00E945E0368EE73E080E090E00E94FA0108958DE061E00E944D
:20036000C10208951F920F920FB60F9211242F933F938F939F93AF93BF9380912E01909153
:200380002F01A0913001B0913101309132010196A11DB11D232F2D5F2D3720F02D570196D4
:2003A000A11DB11D2093320180932E0190932F01A0933001B093310180912A0190912B01D4
:2003C000A0912C01B0912D010196A11DB11D80932A0190932B01A0932C01B0932D01BF917F
:2003E000AF919F918F913F912F910F900FBE0F901F9018959B01AC017FB7F89480912A012F
:2004000090912B01A0912C01B0912D0166B5A89B05C06F3F19F00196A11DB11D7FBFBA2F9E
:20042000A92F982F8827860F911DA11DB11D62E0880F991FAA1FBB1F6A95D1F7BC012DC0FA
:20044000FFB7F89480912A0190912B01A0912C01B0912D01E6B5A89B05C0EF3F19F0019693
:20046000A11DB11DFFBFBA2FA92F982F88278E0F911DA11DB11DE2E0880F991FAA1FBB1F70
:20048000EA95D1F7861B970B885E9340C8F2215030404040504068517C4F21153105410538
:2004A000510571F60895789484B5826084BD84B5816084BD85B5826085BD85B5816085BD64
:2004C000EEE6F0E0808181608083E1E8F0E01082808182608083808181608083E0E8F0E005
:2004E000808181608083E1EBF0E0808184608083E0EBF0E0808181608083E1E9F0E0808178
:2005000082608083808181608083E0E9F0E080818160808320EC30E0F90180818068808391
:2005200080818F7B8083A2ECB0E08C9188608C938C918B7F8C93E1ECF0E0808184608083A0
:20054000808182608083808181608083E3ECF0E0808181608083F9018081826080838C914F
:2005600081608C93EAE7F0E08081846080838081826080838081816080838081806880833B
:200580000895CF93DF93482F50E0CA018C509F4FFC0134914A525F4FFA018491882369F18D
:2005A00090E0880F991FFC01E455FF4FA591B491FC01E654FF4FC591D491662351F42FB789
:2005C000F8948C91932F909589238C93888189230BC0623061F42FB7F8948C91932F9095E3
:2005E00089238C938881832B88832FBF06C09FB7F8948C91832B8C939FBFDF91CF91089523
:200600008730C1F1883080F48330F9F0843030F4813029F1823009F050C024C08430C9F0FA
:20062000863009F04AC022C08A3091F18B3030F4883031F1893009F040C026C08C3091F154
:200640008C3060F18E30C9F533C0809180008F7703C0809180008F7D80938000089584B5BE
:200660008F7702C084B58F7D84BD08958091B0008F7703C08091B0008F7D8093B0000895D8
:20068000809190008F7707C0809190008F7D03C080919000877F8093900008958091C000C4
:2006A0008F7703C08091C0008F7D8093C00008958091C200877F8093C2000895FF920F93A6
:2006C0001F93F62E482F50E0CA018E5E9E4FFC012491CA018C509F4FFC0114914A525F4FC6
:2006E000FA0104910023C9F0222319F0822F0E940003E02FF0E0EE0FFF1FE654FF4FA59132
:20070000B4919FB7F894FF2021F48C911095812302C08C91812B8C939FBF1F910F91FF9031
:200720000895CF93DF930E9453028BE391E00E9458040E94AD01C0E0D0E00E9498012097E2
:20074000E1F30E940000F9CF282F809135018823C1F057FF1AC015C0289890933401809133
:20076000F1008193E217F307B9F74115510539F08091F200882319F48BE68093E800AFBF67
:2007800002C04FEF5FEFCA010895AFB7F89427702093E9008091F200282F30E0241735079D
:2007A0000CF4A901FB019B01240F311D94E6DACFDF93CF930F92CDB7DEB7BE016F5F7F4F6A
:2007C00041E050E00E94A403019719F02FEF3FEF03C08981282F30E0C9010F90CF91DF9125
:2007E0000895FF920F931F93F82E142F052F4091380150913901212F302FC901DC01FB0163
:200800006EEF29C0F7FE02C0949101C09081209136013091370124173507ACF48091E800F3
:200820008570E1F38091E80082FF03C02FEF3FEF17C09093F100C90101968F739070892B64
:2008400011F46093E8002F5F3F4F3093370120933601119731961097A9F6812F902F9C01F6
:20086000C9011F910F91FF9008959C018091E80082FFFCCFF901260F311D03C08091F1000E
:200880008193E217F307D1F7289884E6809334018BEF8093E800CB0108958093E90080912C
:2008A000F200882319F08AE38093E800089508951092350181E08093D70080EA8093D80078
:2008C00082E189BD09B400FEFDCF61E070E080E090E00E94FA0180E98093D8008CE0809317
:2008E000E2001092E000559A209A08955F926F927F928F929F92AF92BF92CF92DF92EF9214
:20090000FF920F931F93CF93DF93E82E842E752E80913501882371F18B01242F352FC90152
:20092000EC017AEFF72E67E0962E9E2050E4552E8E2D90E040E2A42EB12CA822B9223AE3FE
:20094000632E20E4C22ED12CC822D92258C09FB7F8949092E9008091E80085FD02C020E0EE
:2009600004C08091F200252D281B9FBF222361F4FA9419F42FEF3FEF4DC061E070E080E03E
:2009800090E00E94FA013BC0822F90E0C817D9070CF42C2FC21BD1094FB7F8949092E900C0
:2009A000A114B10421F406C01092F10021502223D9F719C0E7FC03C0F801922F10C0C80107
:2009C000322F06C0FC010196E491E093F10031503323C1F706C081918093F100915099237B
:2009E000D1F7020F111D8091E80085FF05C0209729F4C114D10411F06092E8004FBF209790
:200A000009F0A5CF5D9884E680933301282D372DC9019C01C901DF91CF911F910F91FF902A
:200A2000EF90DF90CF90BF90AF909F908F907F906F905F9008951F920F920FB60F92112406
:200A40001F932F933F934F935F936F937F938F939F93AF93BF93EF93FF938091E1001092D8
:200A6000E100982F83FF0FC01092E90081E08093EB001092EC0082E38093ED0010923501C8
:200A800088E08093F00092FF36C083E08093E9008091F200882349F08AE38093E80005C0F1
:200AA00080E891E00E947C0701C012E09FB7F8941093E9008091F2009FBF882389F780917A
:200AC0003301882351F08091330181508093330180913301882309F45D9A809134018823C4
:200AE00051F08091340181508093340180913401882309F4289AFF91EF91BF91AF919F91D6
:200B00008F917F916F915F914F913F912F911F910F900FBE0F901F9018950F931F93DF9368
:200B2000CF930F92CDB7DEB719828E010F5F1F4FC8010E949B07C8010E943409898190E064
:200B40000F90CF91DF911F910F9108951F920F920FB60F921124EF92FF921F932F933F93F4
:200B60004F935F936F937F938F939F93AF93BF93EF93FF93DF93CF93CDB7DEB76197DEBF0F
:200B8000CDBF1092E9008091E80083FF0FC1FE0131969E01275F3F4F03C08091F1008193A1
:200BA000E217F307D1F7289884E68093340182EF8093E800998197FF05C08091E80080FFAF
:200BC000FCCF03C08EEF8093E800292F30E0C90180769070892B09F0C2C08A81882329F4E5
:200BE0001092F1001092F100D6C0813009F4D3C0833009F4D0C0853049F48091E80080FF4E
:200C0000FCCF8B8180688093E300C5C0863009F07CC01C81EF80F8841230C1F51092E900A4
:200C2000109237011092360110923901109238010E948D0599E0FE013996DF01292F1D92E8
:200C40002A95E9F799871A8791E09E8790E8988B9AEF998B2091360130913701275F3F4F61
:200C60003C872B878D871092E9001092370110923601F0923901E092380180E0BF0149E0FD
:200C800050E00E94F1030E948D0585C01092E9001092370110923601F0923901E092380170
:200CA000123241F482E290E00E942C09892B09F476C071C0113079F488E0E816F10419F4E2
:200CC00081E080933A0180913A01882309F06BC0ECE6F1E013C0133009F061C08B818823C0
:200CE00019F4EEE2F1E00AC0823019F4E2E3F1E005C0813009F053C0E4E5F1E0449180E8CE
:200D0000BF0150E00E94F10346C0873009F447C0883021F481E08093F1003DC08930D9F5D6
:200D200023703070232BD9F5E1E9F1E091E031E026E39093E9003093EB0084918093EC0070
:200D40002093ED009F5F3196953099F78EE78093EA001092EA008B81809335011CC08F819A
:200D600098851092E900109237011092360190933901809338018D81882329F4CE01019633
:200D80000E94A70706C0823051F4CE0101960E94FD07882321F08EEF8093E80007C081E2DC
:200DA0008093EB0003C0EEE7F1E0A8CF6196DEBFCDBFCF91DF91FF91EF91BF91AF919F9195
:200DC0008F917F916F915F914F913F912F911F91FF90EF900F900FBE0F901F9018952091AD
:200DE0007C0130917D0180917E0190917F01281B390B2F733070C901089520917C013091E7
:200E00007D0180917E0190917F012817390719F42FEF3FEF09C0E0917E01F0917F01E45C51
:200E2000FE4F8081282F30E0C901089520917C0130917D0180917E0190917F012817390779
:200E400019F42FEF3FEF13C0E0917E01F0917F01E45CFE4F208180917E0190917F0101967F
:200E60008F73907090937F0180937E0130E0C9010895109283011092820188EE93E0A0E010
:200E8000B0E08093840190938501A0938601B09387018EE091E09093810180938001089547
:200EA0000F931F93DF93CF930F92CDB7DEB78C01698380910701882369F083E0BE016F5FCA
:200EC0007F4F41E050E00E9476041816190614F49C0107C081E090E0F8019383828320E039
:200EE00030E0C9010F90CF91DF911F910F91089583E00E944D04089582E00E94D803482F73
:200F000020917C0130917D012F5F3F4F2F73307080917E0190917F012817390759F0E0919C
:200F20007C01F0917D01E45CFE4F408330937D0120937C010895FC0180818E5F808380E881
:200F400065E971E042E450E00E94F1030895FC0181819081913A59F4813209F04CC080E029
:200F600060E071E047E050E00E94F10342C0913209F041C0803239F480E091E067E070E0ED
:200F80000E94350436C0823209F035C08281809307018091000190910101A0910201B09116
:200FA0000301805B9440A040B04019F58091070180FD12C087E797E79093010A8093000A01
:200FC0002BE088E190E00FB6F894A895809360000FBE209360000DC088E10FB6F8948093B2
:200FE0006000109260000FBEA8951092010A1092000A81E0089580E00895FC019181808121
:20100000813A31F4913089F080E0933089F40DC0813269F49B3021F482818093080105C075
:201020009A3029F482818093090181E0089580E00895EF92FF920F931F938C01E62EDC01CA
:20104000ED91FC910480F581E02D0995F82ED801ED91FC910680F781E02DC8016E2D0995C9
:201060008F2D90E01F910F91FF90EF90089510928E01109292011092910180E291E09093B9
:20108000900180938F010895EF92FF920F931F93DF93CF930F92CDB7DEB789838B017A0178
:2010A00084E0BE016F5F7F4F41E050E00E94760484E4B801A7010E9476040F90CF91DF91B0
:2010C0001F910F91FF90EF90089582E048E050E00E9444080895FC01168217821086118675
:2010E0001286138614823496BF010E9465080895DC01683810F0685829C0E62FF0E067FF82
:2011000013C0E058F04081E090E002C0880F991FEA95E2F7809514962C911497282314963E
:201120002C93149760E012C0EB5AFD4F6491662319F420E030E01DC067FF08C014968C9135
:2011400014978D7F14968C9314976F77FD0190E0662321F08681861709F416829F5F319678
:201160009630B1F7CD011496BD010E94650821E030E0C9010895CF93DF93DC01683810F0F3
:20118000685825C0E62FF0E067FF12C0E058F04081E090E002C0880F991FEA95E2F7149641
:2011A0002C911497282B14962C93149760E00FC0EB5AFD4F64916623D9F167FF08C01496A0
:2011C0008C911497826014968C9314976F7716968C9116978617A9F117968C911797861749
:2011E00081F118968C911897861759F119968C911997861731F11A968C911A97861709F1CC
:201200001B968C911B978617E1F0ED01E0E0F0E09E2F8E81882321F4EA0FFB1F668306C004
:201220009F5F31962196E630F10591F7963049F481E090E013969C938E93129720E030E018
:2012400007C0CD011496BD010E94650821E030E0C901DF91CF91089580E867ED71E045E602
:2012600050E00E94F1030895FC0180818F5F808380E86CE372E049E150E00E94F103089586
:20128000CF92DF92EF92FF920F931F93CF93DF937C016B018A01C0E0D0E00FC0D6016D91DA
:2012A0006D01D701ED91FC910190F081E02DC7010995C80FD91F015010400115110571F764
:2012C000CE01DF91CF911F910F91FF90EF90DF90CF900895EE0FFF1F0590F491E02D0994C7
:2012E000F894FFCF00E100000000000001010000000050074009EF061607FD0678077C07FA
:201300000000000019084009BB0878086B08FFFFFFFFFFFFFFFFFFFFFFFFFFFFFFFFFFFFBF
:20132000FFFFFFFFFFFFFFFFFFFFFFFFFFFFFFFFFFFFFFFFFFFFFFFFFFFFFFFFFFFFFFFFCD
:20134000FFFFFFFFFFFFFFFFFFFFFFFFFFFFFFFFFFFFFFFFFFFFFFFFFFFFFFFFFFFFFFFFAD
:20136000FFFFFFFFFFFFFFFFFFFFFFFFFFFFFFFFFFFFFFFFFFFFFFFFFFFFFFFFFFFFFFFF8D
:20138000FFFFFFFFFFFFFFFFFFFFFFFFFFFFFFFFFFFFFFFFFFFFFFFFFFFFFFFFFFFFFFFF6D
:2070000055C000006EC000006CC000006AC0000068C0000066C0000064C0000062C0000043
:2070200060C000005EC00000F1C400005AC0000058C0000056C0000054C0000052C00000EF
:2070400050C0000078C000004CC000004AC0000048C0000046C0000044C0000042C00000BE
:2070600040C000003EC000003CC000003AC0000038C0000036C0000034C0000032C0000048
:2070800030C000002EC000002CC000002AC0000028C0000026C0000024C0000022C00000A8
:2070A00020C000001EC000001CC0000011241FBECFEFDAE0DEBFCDBF11E0A0E0B1E0E0E3BE
:2070C000FFE702C005900D92A83AB107D9F711E0A8EAB1E001C01D92AE3BB107E1F78FD30B
:2070E00025C78ECFF89410926F0010928100109285001092840081E085BF15BE47985D9AEC
:20710000289A0C94000008952091B2013091B3012F5F3F4F3093B3012093B201932F37FFA6
:2071200003C08EEF831B982F990F921710F447980895479A08951F920F920FB60F9211246E
:207140002F938F939F93EF93FF9310928500109284008091A8019091A901009741F00197D3
:207160009093A9018093A801892B09F45D9A8091AA019091AB01009741F001979093AB0126
:207180008093AA01892B09F4289AE0E0F0E0859194918F5F9F4F49F08091AC019091AD0151
:2071A00001969093AD018093AC01FF91EF919F918F912F910F900FBE0F901F90189584E0BC
:2071C0008093E9000DC08091E8008B778093E80003C08EB3882351F08091E80082FFF9CFBE
:2071E0008091E80085FFEFCF8091F1000895982F83E08093E9008091E80085FD0DC0809136
:20720000E8008E778093E80003C08EB3882369F08091E80080FFF9CF9093F1005D9884E6CB
:2072200090E09093A9018093A80108954F925F926F927F928F929F92AF92BF92CF92DF921E
:20724000EF92FF920F931F93CF93DF9384E08093E9008091E80082FF57C2289884E690E067
:207260009093AB018093AA01AADF182F853481F48CE49DE19093AD018093AC0107B600FC4B
:20728000FDCFF999FECF81E180935700E89503C0843519F494DF8DE00DC28C34E1F38035F9
:2072A000D1F3843721F484E4A2DF80E003C2813611F489E5FFC18134B1F481DF182F7FDFE3
:2072C00090E0880F991FAA2797FDA095BA2F312F330F20E0442737FD4095542F822B932B68
:2072E000A42BB52BB8C1803711F483E5E3C1833549F4C0E0D1E089917ADF21E0C730D20714
:20730000D1F7D9C1863521F481E371DF80E3D2C1833731F487E86BDF85E969DF8EE1CAC149
:207320008536B9F4E0E0F0E093E085E090935700E89507B600FCFDCF80935700E89507B65D
:2073400000FCFDCFE058FF4FA0E7E030FA0771F7A2CF823739F4E1E0F0E089E08093570024
:207360008491A8C1863439F4E0E0F0E089E08093570084919FC18E3439F4E3E0F0E089E0E5
:2073800080935700849196C1813539F4E2E0F0E089E08093570084918DC1823631F489E521
:2073A00026DF80E024DF80E885C1823419F0873609F0E5C01092AD011092AC0100DF082FE8
:2073C000FEDEF82EFCDE682E8554823008F071C1902F80E0CF2DD0E0C82BD92B10926F00B3
:2073E000173609F04BC081E180935700E895DD24CC24C3943FC0E090AE01F090AF010091CC
:20740000B0011091B101B6E46B16D9F4ED2DF0E0EE29FF29E4918E2FEADEDD2081F082E08D
:2074200090E0A0E0B0E0E80EF91E0A1F1B1FE092AE01F092AF010093B0011093B101DC2470
:2074400018C0D801C701B695A7959795879558D5CEDE82E090E0A0E0B0E0E80EF91E0A1FF3
:207460001B1FE092AE01F092AF010093B0011093B1012197209709F0BECF7DC08090AE01F5
:207480009090AF01A090B001B090B10196E4691609F05DC083E0F40180935700E89507B63E
:2074A00000FCFDCF54C0F6E46F1661F5772031F1E090AE01F090AF010091B0011091B1019E
:2074C0007EDED82ECC24852D90E08C299D29F7010C0140925700E895112482E090E0A0E08B
:2074E000B0E0E80EF91E0A1F1B1FE092AE01F092AF010093B0011093B10102C060DE582E1A
:20750000742423C0E090AE01F090AF010091B0011091B10116950795F794E79450DE682FFA
:20752000C701F6D48091AE019091AF01A091B001B091B1010296A11DB11D8093AE0190934A
:20754000AF01A093B001B093B101219704C05524772444244394209709F0A5CF96E46916B6
:2075600041F485E0F40180935700E89507B600FCFDCF8DE03CDE82E080936F009CC0833492
:2075800071F40091AE011091AF0119DE90E021E0F8010C0120935700E89511247CCE8336C8
:2075A00019F5E090AE01F090AF010091B0011091B10105DEF701E16090E021E00C0120938C
:2075C0005700E895112482E090E0A0E0B0E0E80EF91E0A1F1B1FE092AE01F092AF0100936A
:2075E000B0011093B10157CE8D3661F4E091AE01F091AF0185E080935700E89507B600FCF2
:20760000FDCF49CE823551F4E091AE01F091AF0105911491812FEBDD802F4CC0843421F5FE
:20762000E090AE01F090AF010091B0011091B10116950795F794E794C2DD682FC70168D4DF
:207640008091AE019091AF01A091B001B091B1010296A11DB11D8093AE019093AF01A093D8
:20766000B001B093B10117CE843609F5E090AE01F090AF010091B0011091B101D801C70142
:20768000B695A795979587953BD4B1DD82E090E0A0E0B0E0E80EF91E0A1F1B1FE092AE010B
:2076A000F092AF010093B0011093B10104C08B3111F08FE39CDD83E08093E9009091E8002B
:2076C0008091E8008E778093E80095FF04C010C08EB38823C9F08091E80080FFF9CF809193
:2076E000E8008E778093E80003C08EB3882361F08091E80080FFF9CF84E08093E9008091F1
:20770000E8008B778093E800DF91CF911F910F91FF90EF90DF90CF90BF90AF909F908F90AC
:207720007F906F905F904F9008959091B601892F8F77813249F58091B7018032A1F081328A
:2077400019F5913A09F58091E800877F8093E8008DE091E067E070E00AD28091E8008B770C
:207760008093E8000895913279F48091E800877F8093E8008DE091E067E070E05CD2809193
:20778000E8008E778093E800089582E061EC42E0B4D083E061E842E1B0D084E060E842E1F1
:2077A000ACC084B7877F84BF88E10FB6F89480936000109260000FBE20E880E090E00FB640
:2077C000F89420936100809361000FBE81E085BF92E095BF3F9A209A559AE1E6F0E02083A1
:2077E000108247985D9A289A109289008AEF8093880090936F0083E080938100EFC01F9336
:2078000088E10FB6F89480936000109260000FBE84B714BE182F10FF08C0E0E0F0E085919B
:2078200094918F5F9F4F09F05DDC2091000A3091010A1092010A1092000A13FF0FC0809143
:20784000090190910A012817390741F0E0E0F0E0859194918F5F9F4F09F044DCA2DF7894F5
:207860001092AD011092AC010CC0E0DC37D38091AC019091AD0181549F4110F010921401DE
:2078800043DC80911401882381F78091E00081608093E00027DC80E090E01F910895FA01A0
:2078A000923049F0933061F09130F9F485E191E022E130E01EC087E291E02EE330E019C06F
:2078C000882329F485E691E024E030E012C0813029F489E691E022E230E00BC0823029F4C2
:2078E0008DE891E028E130E004C080E090E020E030E091838083C90108958093E90080915A
:20790000EB0081608093EB001092ED006093EC004093ED008091EE00881F8827881F0895D6
:207920008091B60188238CF403C08EB38823B1F08091E80082FFF9CF8091E8008B778093B4
:20794000E80008958EB3882349F08091E80080FFF9CF8091E8008E778093E8000895EF9226
:20796000FF920F931F9345D04CD008ED10E0F80180818F77808380818068808380818F7D10
:20798000808319BC1EBA1092B40180EEE82EF12CF70180818B7F8083F8018081816080835B
:2079A00080E060E042E0A9DFE1EEF0E080818E7F8083E2EEF0E0808181608083808188605F
:2079C0008083F70180818E7F8083F8018081806180831F910F91FF90EF900895E7EDF0E01E
:2079E0008081816080838AE482BF81E08093B501B6CFE8EDF0E080818E7F80831092E2000A
:207A000008951092DA001092E10008951F920F920FB60F9211242F933F934F935F936F93D6
:207A20007F938F939F93AF93BF93EF93FF938091DA0080FF1BC08091D80080FF17C08091A3
:207A4000DA008E7F8093DA008091D90080FF0BC080E189BD82E189BD09B400FEFDCF81E0E6
:207A60008EBB3BD203C019BC1EBA37D28091E10080FF17C08091E20080FF13C08091E200B7
:207A80008E7F8093E2008091E20080618093E2008091D80080628093D80019BC85E08EBBE2
:207AA0001CD28091E10084FF2CC08091E20084FF28C080E189BD82E189BD09B400FEFDCF42
:207AC0008091D8008F7D8093D8008091E1008F7E8093E1008091E2008F7E8093E2008091CD
:207AE000E20081608093E2008091B401882331F48091E30087FD02C081E001C084E08EBB2F
:207B0000ECD18091E10083FF21C08091E20083FF1DC08091E100877F8093E10082E08EBB6A
:207B20001092B4018091E1008E7F8093E1008091E2008E7F8093E2008091E200806180931F
:207B4000E20080E060E042E0D8DEC7D1FF91EF91BF91AF919F918F917F916F915F914F9163
:207B60003F912F910F900FBE0F901F9018959C014091BC015091BD014617570718F4F90183
:207B800090E044C06115710511F0AB01F8CF8091E8008E778093E80040E050E0F0CF8EB3C8
:207BA000882309F444C0853009F443C08091E80083FF02C081E008958091E80082FD31C0C0
:207BC0008091E80080FF22C08091F3009091F200782F60E0292F30E0262B372B07C0819159
:207BE0008093F100415050402F5F3F4F4115510519F02830310598F390E02830310509F47B
:207C000091E08091E8008E778093E8004115510531F6992321F605C08EB3882341F08530BD
:207C200041F08091E80082FFF7CF80E0089582E0089583E008959C016115710529F4809120
:207C4000E8008B778093E800F90126C08EB3882391F1853091F18091E80083FF02C081E01C
:207C600008958091E80082FFF1CF06C08091F10081936150704059F02091F3008091F20000
:207C8000322F20E090E0822B932B892B79F78091E8008B778093E80061157105B9F605C02E
:207CA0008EB3882341F0853041F08091E80080FFF7CF80E0089582E0089583E008950F93E5
:207CC0001F93DF93CF9300D0CDB7DEB7E6EBF1E08091F100819381E0EE3BF807C9F725DD32
:207CE0008091E80083FFE4C08091B6019091B701953009F46DC0963040F4913081F19130E7
:207D000070F0933009F0D4C02AC0983009F4A3C0993009F4B2C0963009F0CAC07CC080382C
:207D200009F4C6C0823809F0C3C08091BA0187708093E9008091EB001092E9002091E800AB
:207D4000277F2093E80090E025E0969587952A95E1F781708093F1001092F10087C0882315
:207D600019F0823009F0A4C08F71823009F0A0C08091B801882331F52091BA01277009F445
:207D800097C02093E9008091EB0080FF1BC0933021F48091EB00806213C08091EB00806134
:207DA0008093EB0081E090E002C0880F991F2A95E2F78093EA001092EA008091EB008860DE
:207DC0008093EB001092E9008091E800877F51C0882309F06DC01091B8011F770FB7F894F7
:207DE0008091E800877F8093E8009ADD8091E80080FFFCCF8091E3008078812B8093E30041
:207E000080688093E300112311F482E001C083E08EBB0FBF4DC08058823008F049C0809105
:207E2000B8019091B9016091BA01AE014F5F5F4F36DDBC01009709F43BC08091E800877F99
:207E40008093E80089819A8192DE8091E8008B778093E8002DC0803859F58091E800877FAA
:207E60008093E8008091B4018093F1008091E8008E778093E80054DD1BC08823C9F49091AF
:207E8000B8019230A8F48091E800877F8093E8009093B40145DD8091B401882331F4809130
:207EA000E30087FD02C081E001C084E08EBB6DDC8091E80083FF0AC08091EB00806280934B
:207EC000EB008091E800877F8093E8000F900F90CF91DF911F910F91089508951F938EB332
:207EE000882361F01091E9001092E9008091E80083FF01C0E4DE17701093E9001F91089513
:207F0000F999FECF92BD81BDF89A992780B50895262FF999FECF1FBA92BD81BD20BD0FB695
:207F2000F894FA9AF99A0FBE01960895F894FFCF4341544552494E41007777000A000000F4
:207F4000000000080112011001020000084123350001000201000109023E0002010080324E
:207F60000904000001020201000524001001042402040524060001070582030800FF0904B1
:207F80000100020A00000007050402100001070583021000010403090422034100720064BF
:207FA00000750069006E006F0020004D006900630072006F00200020002000000018034130
:187FC0000072006400750069006E006F0020004C004C0043000000001D
:00000001FF
